:1000000012C0189592C118951895189518951895BD
:100010001895189518951895189518951895189578
:100020001895189518958FED8DBFC0ECE8EB4E2E06
:10003000DD275D2EEEE7F0E0A0E6B0E088278D93A7
:100040003197E9F783E389B980E082B988E18AB919
:1000500066248C9A94988D9A95988A9A87E088BBA2
:10006000789483E083BF80E080BF85B7837F84601E
:1000700085BF789481E080936600009166000F3020
:1000800010F009F011C0E6E6F0E0A190E1E0F0E048
:10009000EA0DA6E6AD90A6E6AA0D7FD2A6E68C9163
:1000A0008F5F8C9308F4E9CFE1E0F0E0A6E775D22A
:1000B000009176000F3F09F009C080E08093760040
:1000C000E1E0F0E0A6E77BE757D22FC081E0809324
:1000D00065004091760000916500041710F009F06A
:1000E00024C00091650045E062D2A8E74C930091DE
:1000F000780044E0041BA7E70C938091770080937D
:1001000066004091780000916600041710F009F035
:1001100006C0A6E68C918F5F8C9308F4F2CFA5E61B
:100120008C918F5F8C9308F4D4CFA0E6A0938300CA
:10013000B093840029D1082F013009F022C081E05A
:100140008093650000916500053010F009F006C04D
:10015000A5E68C918F5F8C9308F4F4CFEBE7F0E089
:10016000FA93EA93E0E6F0E0FA93EA936CD02496EF
:1001700000917B00003010F009F001C001C0929A9C
:1001800000C0B0995CC0A0E6A0938300B093840047
:10019000FBD0082F013009F051C0E0E1FA93EA9357
:1001A000E0E6F0E0FA93EA934ED02496003009F0AE
:1001B00044C000917600033008F03FC0A6E78C9160
:1001C0008F5F8C93E1E0F0E0A6E77BE7D5D100916B
:1001D000760045E0ECD1A6E64C93A6E68C918450DF
:1001E0008C9381E08093650000916500053010F0EC
:1001F00009F020C0A5E6AD90AFE5AA0D8C91A6E66A
:10020000AD90A6E6AA0D8C93E6E6F0E0A190E1E0C1
:10021000F0E0EA0DA5E6AD90AFE5AA0D7BE7ACD125
:10022000A6E68C918F5F8C93A5E68C918F5F8C9363
:1002300008F4DACF88EE93E098D001C0A4CF84EF21
:1002400091E093D072CF81E08093790000917900A2
:10025000053010F009F015C0A0EAB0E0E9E7F0E0E1
:10026000A190E881F981EA0D319766D160D0E6EC82
:10027000F5E065D06AD0A9E78C918F5F8C9308F484
:10028000E5CF81E08093790000917900033010F090
:1002900009F046C00091790045E089D1A8E74C9368
:1002A0000091780044E0041BA7E70C9380E0809362
:1002B0007A008091770080936600409178000091E9
:1002C0006600041710F009F01AC0AAE78C918F5F3E
:1002D0008C93AAE7AD90A881B981AA0D11974C9192
:1002E000A6E6AD90A6E6AA0D0C91041709F401C08C
:1002F00006C0A6E68C918F5F8C9308F4DECF009148
:100300007A00053009F006C080917900AA81BB818E
:100310008C930AC0A9E78C918F5F8C9308F4B4CFBB
:1003200080E0AA81BB818C93089552D01895A0EAF1
:10033000B0E08D91882311F00BD0FBCF0895F8D059
:10034000802D11F005D0FBCF08958DE001D08AE01B
:100350005D9BFECF8CB908953197F1F708956894AD
:1003600062F80895E89462F80895EF93FF93EE27FA
:10037000E82BE92B31F0E0EDF7E03197F1F7019749
:10038000D1F7FF91EF91089519D08BB780688BBF9B
:100390009091810088B781FF05C0816088BF9A95E0
:1003A00090938100903021F080917C00803081F327
:1003B0008BB78F778BBF80917C00089584E6809304
:1003C00081008827ACE795E08D939A95E9F7089529
:1003D0008F938FB78F930F931F932F933F934F93C9
:1003E0005F936F937F939F93AF93BF9330B33870B6
:1003F00098E0392709F031E0009152001091820015
:10040000202F211B203308F458C0009382009091C4
:100410007D00913090F4313011F0D3DF4EC09091D7
:100420007E00939590937E00993009F046C03093FA
:100430007D00992790937E0040C0923089F1909181
:100440007E00939590937E0000918000030F0093AF
:100450008000953089F400FF02C0B3DF2EC0002772
:100460000093800000937E0090917F00983229F5E0
:1004700092E090937D0021C090917F00939590939E
:100480007F003795A0918300B09184008C91881FE4
:100490008D9304E08C91881F8D930A95D9F70DC038
:1004A00090917F00939590937F0037958091800085
:1004B000881F809380009D3279F0BF91AF919F910A
:1004C0007F916F915F914F913F912F911F910F916C
:1004D0008F918FBF8F910895082F079541E008F401
:1004E000ECCF14E0A0918300B091840095E0222726
:1004F000542F550F550F550F550F642F752F8D9194
:10050000782309F071E0682309F061E026272727A6
:100510009A9571F70024079508F40394021609F0E0
:10052000CCCF440F1A95F1F681E080937C00C5CFC3
:10053000C89531960020089541E003C042E001C013
:1005400044E0E40F8827F81F8291982F829505D008
:10055000892F03D04A95C1F707C08F708A3008F001
:10056000895F805D8D93089588278D930895E19923
:10057000FECFEEBB3196089591E001C092E07B374B
:1005800051F47FB7F894F3DF8D918DBBE29AE19A35
:100590009A95C9F77FBF7727089591E001C092E04F
:1005A000E6DFE09A8DB38D939A95D1F70895FF9386
:1005B0005527F8E0469508F4500F57954795FA955A
:0805C000D1F7FF9108952C0012
:00000001FF
